:100000006F10907E1300000013000000130000002A
:100010001300000013000000130000001300000094
:100020001300000013000000130000001300000084
:08003000130000007300100032
:1000380000000000000000007C1F00007E1F000080
:1000480000000000801F0000000000000000000009
:10005800821F0000841F0000000000000000000054
:100068003827000000000000881F00000000000082
:100078008A1F00008C1F00008E1F0000901F0000C8
:10008800921F0000941F0000961F0000981F000098
:100098009A1F00009C1F00009E1F0000A01F000068
:1000A800A21F0000A41F0000A61F0000A81F000038
:1000B800AA1F0000AC1F0000AE1F0000B01F000008
:1000C8004E270000B41F0000B61F0000B81F000034
:1000D800BA1F0000BC1F0000BE1F0000C01F0000A8
:1000E800C21F0000C41F0000C61F0000C81F000078
:1000F800CA1F0000CC1F0000CE1F0000D01F000048
:10010800D21F0000D41F0000D61F0000D81F000017
:10011800DA1F0000DC1F000056270000E01F000067
:10012800E21F0000E41F0000E61F000000000000BE
:080138000000000000000000BF
:10014000397101436EC619A0397141536AC866CA34
:1001500062CC5ECE19A0397101535AD056D252D416
:100160004ED64AD826DA22DC06DE3301614082828E
:1001700041114AC026C222C406C68282B24D410144
:10018000024D924C224CB24B4101024B924A224A00
:10019000B2494101024992442244B2404101828065
:1001A0003D432A876373C3029377F700BDEFADE544
:1001B000937606FF3D8ABA960CC34CC30CC74CC756
:1001C0004107E36BD7FE11E28280B306C3408A0683
:1001D0009702000096966780A6002307B700A30643
:1001E000B7002306B700A305B7002305B700A30493
:1001F000B7002304B700A303B7002303B700A3028B
:10020000B7002302B700A301B7002301B700A30082
:10021000B7002300B700828093F5F50F9396850011
:10022000D58D93960501D58D61B7939627009702DA
:10023000000096968682E78086FA9680C1171D8F09
:100240003E96E374C3F8A5B7EFF29FF2B70500201E
:100250009385051BEF00D07535BFEFF27FF19385D5
:100260008180EF00F0743DB78280B70700201387CC
:10027000C7778567BA9705472398E7848280EFF2AE
:100280003FEF9385E1610D45EF10104D420541812F
:10029000B70700201387C7778567BA972399A78880
:1002A0000547239AE788FDB5EFF29FEC0111B76788
:1002B000004003A747C4420741839387C1879AA39D
:1002C0009E2303D7418AF98F93F7072099CF376789
:1002D0000040C1679387F7DF2322F7C413870187A4
:1002E0001C23850793F7F70F1CA383D7C18703D778
:1002F000418AF98FC207C18763CF070A83D7C187B5
:1003000003D7418AF98F93F7074089CF37670040B9
:10031000C1679387F7BF2322F7C4B707002083A7DD
:100320004712829783D7C18703D7418AF98F1397E2
:1003300027016358070037670040B967FD1723227C
:10034000F7C483D7C18703D7418AF98F1397370141
:100350006346070683D7C18703D7418AF98F13976E
:100360004701635E070083A78183BDC3EF00007C64
:1003700037670040BD679387F77F2322F7C483D791
:10038000C18703D7418AF98F93F707109DC3376759
:100390000040C1679387F7EF2322F7C4832787C400
:1003A00013970701634A070223AA01861D45EF0040
:1003B00070070561C5B3EF10A03A89B737670040F1
:1003C000BD67FD172322F7C40145EF00B00559B7FB
:1003D0000945EF00300569BF9387418798430507BA
:1003E00098C398438D47E3F3E7FCB767004083A7C2
:1003F00007C4A18BC5FF37660040832706C4C20728
:10040000C18323ACF186130606C08147C165FD1583
:1004100021451442ED8E13972700130801024297DD
:100420002320D7FE85071106E395A7FE93878187D2
:1004300098431367170098C3944341677D17F98E5B
:10044000376600402320D6C49443F99A94C39C4352
:100450007D8F2320E6C437670040832747C493F786
:100460000740E5DFB7660040C1679387F7BF23A267
:10047000F6C4938606C0814741667D16A145139751
:10048000270008102A97032707FE718F98C2850757
:100490009106E396B7FE23AA018609BF03A701864A
:1004A00083A7C1856319F70083C7818593F7F70F89
:1004B000014591E38280EFF2BFCB138401861C409B
:1004C0009384818698401A079A07938501ACBA9560
:1004D0001385018C3E95EF2040799C4013971700BF
:1004E000938701CCBA978AA31C40138797FF85078F
:1004F0003337E0003307E040F98F138701861CC3D0
:10050000184383A7C185630BF70283C7018193F763
:10051000F70F85EB83A78186138797FF850733370E
:10052000E0003307E040F98F138781861CC318432E
:1005300083A7C1860545630FF702A9B9238C0184FF
:10054000E9B7238801809387818698439C439396DB
:100550001700938701CCB6971A079223938501ACB5
:10056000BA9513051008EF10901C0545EF10E079BF
:100570000545E1B705472382E186C1B718219D47AC
:100580006308F70403A7C18583A701866317F700F3
:1005900083C7818593F7F70FB9E7EFF27FBD2E860A
:1005A000AA851384C1851C409A071385018C3E954A
:1005B000EF50A0621C4085071CC01840A147630D86
:1005C000F70003A7C18583A70186630AF700D9B6A0
:1005D0000547238EE18A828023AE0184DDB705477B
:1005E000238CE184EDB78280EFF29FB83971130656
:1005F000000481450A856D368A850545EF10D015C2
:10060000930500040A859D3F8D650545EF10006A3E
:10061000216149B603A7C18683A781866317F700C6
:1006200083C7418693F7F70FA1CFEFF27FB413840E
:10063000C18618401C4093961700938701CCB6974B
:100640001A079223938501ACBA9513051008EF1091
:10065000100E0545EF10606B1C4085071CC018404C
:10066000A1476309F70003A7C18683A781866306B4
:10067000F7000DB623A60186FDB723820186D5BFFC
:1006800005472388E1808280EFF29FAE613719B67B
:1006900083C7A1CF81C7154723A4E1888280114772
:1006A00023A4E188828082808280828091E58547D0
:1006B00033B5A700060582800945828001C51385F0
:1006C0004184828083A781891D479AAB828001C5BE
:1006D00013854184828083A781891D479AAB8280DC
:1006E000EFF21FA903A781891C2393F7F70785461B
:1006F0006385D7029306100209456399D7041C331A
:1007000013071002638AE704130700026390E704EB
:10071000370400001304E46C15A03C239306200268
:100720006387D7029306100209456391D7023714F5
:100730000000130424AF00CF0145029483A78189F0
:1007400080CF23990700014502940145A1B43714D5
:100750000000130424AEC5B7370400001304C46BB3
:10076000F1BF83A7818998339C2393F7F7079306FA
:10077000100201456383D70082801307E7FD1377DA
:10078000F70F05453335E5000605FDB703A7818959
:100790001C2393F7F707930610026383D700828028
:1007A000183393070002E31CF7FEEFF27F9C1385DA
:1007B0004184EF20E029F9BAEFF29F9B83A781895A
:1007C000238507003D2EB7670040938707C0056665
:1007D0001306F6F0B7660040938606C29843718F01
:1007E00098C39107E39CD7FEB76700401307F00F4B
:1007F00023A2E7C4EF10A07123A40188814501451D
:10080000EF1030765145EF20000285450545EF1089
:1008100050756FF03F98EFF2BF9583A781892385CC
:1008200007001967034737C998B7A3850700014533
:10083000EF10803F930500200145EF10E03F930546
:1008400000080145EF10405B930500040145EF10DF
:10085000A05C37040020130404128345C402014540
:10086000EF1040618345C4020145EF108062C1452D
:100870000145EF10603E8D650145EF102043B767DD
:10088000004083A707C01397170163520702B7669A
:10089000004083A706C0C207C18305671307F7F0AE
:1008A000F98F316713070708D98F23A0F6C0B76700
:1008B000004083A707C093F707048DC3B7660040C5
:1008C00083A706C0C207C18305671307F7F0F98F36
:1008D00021671307070CD98F23A0F6C0930500608A
:1008E0000545EF1060359305000C0545EF10C0502D
:1008F000930500100545EF102052930500040545AF
:10090000EF104057930500040545EF1080589305FC
:1009100000020545EF1040348D650545EF100039A4
:10092000B767004083A747C093F707048DC3B76636
:10093000004083A746C0C207C18305671307F7F0CD
:10094000F98F21671307070CD98F23A2F6C0B76769
:10095000004083A747C01397170163520702B76689
:10096000004083A746C0C207C18305671307F7F09D
:10097000F98F316713070708D98F23A2F6C09305B3
:1009800000600945EF10402B930500140945EF1056
:10099000A046A1450945EF10E04D93050002094529
:1009A000EF10802B81450945EF104030B7670040BC
:1009B00083A747C093F707048DC3B766004083A79A
:1009C00046C0C207C18305671307F7F0F98F216797
:1009D0001307070CD98F23A2F6C081450D45EF10F0
:1009E000A025930500180D45EF1000419305001C4C
:1009F0000D45EF106042930500040D45EF10804750
:100A0000930500040D45EF10C048930500020D4505
:100A1000EF1080248D650D45EF104029B767004029
:100A200083A7C7C093F707048DC3B766004083A7A9
:100A3000C6C0C207C18305671307F7F0F98F2167A6
:100A40001307070CD98F23A6F6C0B767004083A70A
:100A5000C7C01397170163520702B766004083A708
:100A6000C6C0C207C18305671307F7F0F98F316766
:100A700013070708D98F23A6F6C00145EF003040C1
:100A8000854623A4D188B70700201387C7778567D9
:100A9000BA972398D7846FF0EFEFEFF26FED93855D
:100AA000C181EF00E0706FF0EFEEEFF26FEC938535
:100AB0004181EF00E06F6FF0EFED83A78189AC33E8
:100AC000914763EEB700EFF2AFEA8E05B70700205B
:100AD00093870715BE95EF00A06D6FF0AFEB014552
:100AE0008280EFF2EFE893850183EF00606C6FF096
:100AF0006FEAEFF2EFE793858182EF00606B6FF0B2
:100B00006FE9B7670040054723A0E7C423A007C4E7
:100B100023A207C40967130707C02392E18A096764
:100B2000130707C023A0E7C4014582803766004051
:100B3000832506C4C205C181130606C081474168EA
:100B40007D18138501CDA1481442B3F60601139711
:100B500027002A9714C385071106E39717FF13E7A9
:100B60000540B767004023A0E7C413E7154023A062
:100B7000E7C4F999C205C18113E7054023A0E7C482
:100B800037670040832747C493F70740E5DFB76620
:100B90000040C1679387F7BF23A2F6C4938606C0BF
:100BA0008147138501CD41667D16214813972700A3
:100BB0002A971843718F98C285079106E39807FF1B
:100BC00093E58540376700402320B7C4832707C4D7
:100BD000C207C18393E747002320F7C40D4723A42E
:100BE000E188828083C7A1CF89C7154723A4E18804
:100BF0008280054723A4E1888280EFF26FD73764B3
:100C00000040832704C4C207C183ED9BC207C18390
:100C10002320F4C4C13FB167938707F02320F4C4B5
:100C20006FF04FD79D476304F50023A0A18883A7E9
:100C3000018815476363F70CEFF28FD38A071967B2
:100C4000130707D8BA979C43828783A7C18889C7AF
:100C5000154723A0E18829A84D37194723A0E1882B
:100C600001A8613F114723A0E188054723A6E18839
:100C70006FF04FD2938701880947D8A30D4798C3D7
:100C8000C5BF93870188D8237D171377F70FD8A3A3
:100C9000DC2393F7F70FE9FF114723A0E188C9BFD1
:100CA00037670040832707C4C207C18393E7070162
:100CB0002320F7C493870188154798C32947D8A3F1
:100CC00045BF93870188D8237D171377F70FD8A3E3
:100CD000DC2393F7F70FC9FF37670040832707C46A
:100CE000C207C183BD9BC207C1832320F7C4194734
:100CF00023A0E18823A60188A5BF194723A0E18886
:100D0000828001CDEFF2CFC683A7018A9C438297F0
:100D100003A5818929056FF0EFC783A7818905475E
:100D20009AAB828001CDEFF2AFC483A7018A9C47C2
:100D3000829703A5818931056FF0CFC583A781898B
:100D400005479AAB828039C1239A018803A781891C
:100D50001C2393F7F707B1E71C3713F7070201C706
:100D60008946238AD18893F7070495C793874189D9
:100D700098231367170098A3EFF28FBF83A7018A08
:100D80009C4B8297138541896FF0CFC083A78189DF
:100D900009479AAB8280938741899823799B98A3CE
:100DA000E1BF8546638DD70489460145639CD7041E
:100DB00058339377F70062076187634207028A0717
:100DC00037670040130707C0BA979C430D67F98F38
:100DD0000567E393E7FA0547238AE18871BF8A072D
:100DE00037670040130707C0BA979C4393F7070380
:100DF0004147E393E7F80547238AE188B5BF1385A8
:100E0000418982808280EFF20FB583A48189822894
:100E100039E4982491476305F700DE281149A1A021
:100E200003A7018985476307F70041472394E18AB7
:100E30001D49A5A8B767004083A707C5C207C1839E
:100E4000373700200907BA97860723A00700130742
:100E500000032394E18A23A801881149B9A0DE2860
:100E600063FB8704094963F387003E8442044180A1
:100E70009C4C22858297AA890145EF00107C22862E
:100E8000AA854E85EF007056A2850145EF00907E41
:100E90009E28818F9EA8BE283E94A2A81307000317
:100EA0002394E18A0D672393E18A83A781892384B0
:100EB00027016FF08FAD11497DB783A78189B833C2
:100EC00083C65182094563E0E602B42389EED62346
:100ED00099EAEFF2EFA9B8A783A7018ADC438297CA
:100EE00001456FF02FAB8280EFF28FA883A7818935
:100EF00003A7C189184FAC33C833029783A78189F0
:100F0000B82709440DC32A8415E1D82315E3BC236F
:100F100095E383A7018ADC47829783A78189D83329
:100F2000B8B7B833D8A722856FF0CFA60944E5BF7C
:100F30000944D5BF0944C5BF03A781891C2393F782
:100F4000F70791C7894609456389D70082801C3716
:100F500093F7F7FD1CB7014582803E23E5FB5C2338
:100F6000F5F75C3313F6F7F7E207E18763CC070484
:100F700093162600B7650040938505C0AE9694424F
:100F80008D65ED8E83C541820945E371B6FCDDDEDA
:100F900038274DDFEFF2CF9D63C1070413142600FD
:100FA000B7670040938707C03E941C400D67F98FD8
:100FB0000567638CE70483A7018ADC4B82970145B0
:100FC0006FF04F9D93162600B7650040938505C0CE
:100FD000AE96944293F6060375B7931726003767CB
:100FE0000040130707C0BA979C4393F70703414794
:100FF000E393E7FC1374F60F2285EF00105D930571
:1010000000032285EF0050457DB731E6B707002089
:1010100083C5C7140145EF00D0671840F177938767
:10102000F7F87D8F420741838D673D8FE177938786
:1010300007085D8F4207418318C01C408D66F58FFD
:10104000E38BD7F641667D1618C01C40F18FF58FF3
:10105000E39CD7FE8DB73285EF0030541840F1770E
:101060009387F7F87D8F420741838D673D8FE17746
:10107000938707085D8F4207418318C01C408D6627
:10108000F58FE38AD7F241667D1618C01C40F18FB8
:10109000F58FE39CD7FE05B703A681895832937775
:1010A000F7F7620761876347070893962700B765DC
:1010B0000040938505C0AE9694428D65ED8E83C544
:1010C0004182094563F6B70C2E22F9E1F1C23426BC
:1010D000E1C2EFF2EF89634A07068A0737670040EB
:1010E000130707C0BA97944371771307F7F8F98E7F
:1010F000C206C1820567B98E617713070708D98ECA
:10110000C206C18294C398430D66718F0566630C55
:10111000C70041667D160D65856594C39843718F40
:10112000698FE31CB7FE83A7018A9C4F8297014514
:101130006FF04F8693962700B7650040938505C0F2
:10114000AE96944293F606039DBF8A073767004028
:10115000130707C0BA97944365771307F7FBF98E17
:10116000C206C18293C60601617713070708D98EAC
:10117000C206C18294C39843137707034146E30430
:10118000C7FA94C3984313770703E31CC7FE61BFF4
:101190008280EFE2FFFD03A781891C3793E70702F6
:1011A0001CB783A7018ADC4F829701456FE09FFE41
:1011B00083A78189BA2B01C588413A958280CA21CB
:1011C000198D8AAB01458280EFE29FFAB7070020B4
:1011D00083C5C7140145EF00D04B83A781898827B9
:1011E000A1476307F5005D15133515006FE09FFA01
:1011F00005672393E18A41472394E18AEDB7EFE243
:101200003FF74111B767004083A707C503A781894E
:101210001027A5466315D60483A78189054798A79B
:10122000FA2363190712803398231377F70745EBE6
:101230002547630EE4061547630FE4060D47630870
:10124000E40805476313E40AB4336390E60ADA233B
:1012500049EF9C3793F70702C9CBF93999A8416444
:101260009306F4FFF58F373600201106B2978607F4
:101270008043758C0604B76700403E941C201CA375
:1012800083A78189183098B303A981894A20EF0088
:1012900030472311A90003A981890A24EF00504691
:1012A0002312A9005A2483A78189FAA3B5B7EFF0C6
:1012B000DFC039C51DA883863700214763C40606F1
:1012C000B423ADE2D623B9EEBC279DCBA1A8B4339D
:1012D0000547639CE600DE2389EB653DD9BF854762
:1012E0006309F7048947630CF70483A7C189DC4BC2
:1012F000228582978D4725476306F50221471DE128
:10130000B767004083A707C5C207C18337370020EE
:101310000907BA97860723A0070013070003239441
:10132000E18A194783A7818998A7793D41016FE038
:101330007FE6AD47E31BF4FAEFF01FBB9DBF854787
:101340006307F4008D47E312F4FAB9339DB7EFF069
:10135000BFBE85B798339946630FD7046318071249
:10136000BA2311EBD843C1769386F60F758FB70673
:1013700002006300D70803A7818983A7C1899C4B1A
:10138000083382978D476308F51A83A78189962BC6
:1013900041677D176386E61209476303E51A638197
:1013A000061A038707006340071A0D4798A70D67C1
:1013B0002393E18A9DBF98231377F7074DFFBC2342
:1013C0000547638FE70009476381E7023D47638074
:1013D000E71C0D47E391E7FA83A7C189DC5321A0FD
:1013E00083A7C189DC4FC1DB75A883A7C1899C5342
:1013F000DDBF98231377F70701EBDE23ADFFB717A7
:101400000000938767D479A885466312D70203A7A3
:10141000C189184F8145C833029731FD83A781895F
:10142000BC27B1DBB7170000938767D4A5A889460E
:10143000E313D7F4DC3393F6F70013978701618742
:10144000634B07021397260037660040130606C059
:10145000329718430D66718F03C64182E3FDC6F0D3
:1014600093F70707E39907F0E30707F0B7170000C2
:10147000938767D405A813972600376600401306A4
:1014800006C03297184313770703F9B7A146631CC8
:10149000D7029C2393F7F707E39F07ECB7170000E9
:1014A000938727D003A78189231907001CCF014503
:1014B000829783A78189962B41677D17E391E6EE9A
:1014C000254798A79DB5A9466313D704982313779A
:1014D000F7078546E311D7EAB827E30E07E8BA23F2
:1014E000E31B07E8D843C1769386F60F758FC16674
:1014F000E313D7E803A7C189184F8145C833029782
:10150000E31B05E6B7170000938747D261BF94231A
:1015100093F6060613060004E39FC6E49306400311
:10152000E31BD7E4D8339D47E317F7E4B707000080
:101530009387A72585BF83A78189254798A7F5B3FA
:10154000214798A7DDB3FA233AC63246637CD6001A
:1015500032479AAB03A7C1890347C702DAABEFF062
:101560009F8AE1B3E3F8E6FE03A7C1890347C702F8
:1015700013160701418263F5C60023A80188D9BF6D
:10158000B3E6E602E1FA854623A8D188E1B7B707BA
:1015900000009387872439B7EFE29FBD03A48189B8
:1015A00018249307E7FF93F7D70FA146F1C39307DA
:1015B000D7FF93F7D70F99CB9D47A146631AF70A38
:1015C00083A7C189DC478297A1465DA01C4C8DCBC7
:1015D0000628C1C45A2863739700BA84C204C18024
:1015E000268582972A891E28858F1EA83E28A697C1
:1015F0003EA80145EF0030062686AA854A85392592
:101600001E28A1CF0D672393E18A81450145EF0094
:101610007006130700032394E18A1E285A2863F2F8
:10162000E70491C783A78189154798A73DA883A799
:101630008189194798A7B767004083A707C5C207E4
:10164000C183373700200907BA97860723A0070010
:10165000130700032394E18A09A81A285E28E36887
:10166000F7FC83A781890D4798A783A781899427D1
:1016700083A7818994A7EFF03FB56FE0BFB103CE98
:101680004182630F0E02814637630040130303C09B
:10169000C168FD1805681308F8F0A1659385050871
:1016A00013F6F60F131726001A971C43B3F717010A
:1016B000B3F70701D18FCD8F1CC38506E312DEFE81
:1016C00013650508B767004023A6A7C48280EFE230
:1016D0003FAA83A6818998269307E7FF93F7D70F40
:1016E00099CF1946A1476311C70298329547630401
:1016F000F70283A7C1899C478297A14731A0EFF0E9
:101700008FF083A781899C2703A781891CA7EFF00D
:10171000BFAB6FE03FA89C2293F7F707F9FBA83215
:10172000B93F83A7018A9C538297E1B78280EFE299
:101730003FA4938701CF23ACF188094798A73707C7
:1017400000209306071223AED188B70700209387A5
:10175000871723A0F18A8327071282976FE09FA340
:10176000EFE27F9F411123170100B7690040138406
:1017700009C0370A0020130A8A0EB70A0020938A8C
:101780004A10E1A01840420741839387618A9AA3D7
:101790009A23137707032394E18A9A238D66758F22
:1017A0009AA31C4025671307F7FBF98F1840B16611
:1017B0009386F6F8758F8966358F93C707029396DF
:1017C0000701C182D98F216613060608D18F1CC07C
:1017D0001C4093F7070313060002638EC700E177EE
:1017E00093870708DD8EC206C18214C01C4093F7A0
:1017F0000703E39CC7FE1C408D66F58F89666382F4
:10180000D702E177938707085D8F42074183C1665E
:10181000FD168D65096618C01C40F58FED8FE39CA1
:10182000C7FE83D7C187C18BD9C31C40C207C18300
:101830007C873887856793870780F98F639F0716B2
:101840003C87C207C18763CF072683A749C4139784
:1018500007014183239EE18613970701635C071408
:1018600083D7C187BD8B238BF18889DF8A07A29735
:101870009843420741837887388742074187634806
:1018800007343C8793F70708E9D383C761898A0740
:10189000A2979843A5669386F6F0758F98C383C781
:1018A0006189FD178A07D2979C43829779BF376475
:1018B0000040832704C0A5641387F4F0F98F232028
:1018C000F4C03135032704C09384F4FB658F0326ED
:1018D00004C0B1679387F7F87D8E83D7618A9396AA
:1018E000370163D4060085673D8E83D7618A93965E
:1018F000270163D4060089673D8E83D7818AC18B17
:1019000099C31347070183D7818A93F7070299C3C5
:101910001347070293170701C183518FA16693866E
:101920000608558FB766004023A0E6C083A606C010
:1019300003D7818A4207418393F606036388E60250
:10194000E17593850508CD8FB7660040938606C084
:1019500093950701C1818CC298429387818A9E2307
:10196000C207C18313770703E317F7FEB767004089
:1019700003A707C083D7618AC207C1838D66758FAD
:10198000630AF702E177938707085D8EB766004028
:10199000938606C042064182C165FD150D6590C261
:1019A0009C421387618A1A2342074183ED8FE98F96
:1019B000E397E7FE41016FE04FFD37640040832766
:1019C00004C005671307F7F8F98F2320F4C0EFF080
:1019D0001F83832704C025671307F7FBF98F0326AE
:1019E00004C031671307F7F8798E03D7618A93161D
:1019F000370163D406000567398E03D7618A9316D1
:101A0000270163D406000967398E03D7818A418B89
:101A100019C393C7070103D7818A1377070219C334
:101A200093C7070293950701C181D18F21671307DF
:101A30000708D98F376700402320F7C0032707C066
:101A400083D7818AC207C183137707036307F7022D
:101A5000E17793870708DD8DB7660040938606C05F
:101A6000C205C1818CC298429387818A9E23C20796
:101A7000C18313770703E317F7FEB767004003A797
:101A800007C083D7618AC207C1838D66758FE30360
:101A9000F7F2E177938707085D8EB766004093867B
:101AA00006C042064182C165FD150D6590C29C428B
:101AB0001387618A1A2342074183ED8FE98FE397E9
:101AC000E7FECDBD37640040832704C005671307D8
:101AD000F7F8F98F2320F4C0EFF01FAC832704C080
:101AE00025671307F7FBF98F032604C03167130737
:101AF000F7F8798E03D7618A9316370163D406000D
:101B00000567398E03D7618A9316270163D40600CF
:101B10000967398E03D7818A418B19C393C707019F
:101B200003D7818A1377070219C393C707029395D6
:101B30000701C181D18F216713070708D98F376744
:101B400000402320F7C0032707C083D7818AC2073C
:101B5000C183137707036307F702E17793870708C9
:101B6000DD8DB7660040938606C0C205C1818CC278
:101B700098429387818A9E23C207C1831377070304
:101B8000E317F7FEB767004003A707C083D7618A52
:101B9000C207C1838D66758FE30EF7E0E177938707
:101BA00007085D8EB7660040938606C042064182F4
:101BB000C165FD150D6590C29C421387618A1A2389
:101BC00042074183ED8FE98FE397E7FEE5B3984342
:101BD00085669386F6F8758F98C383C76189FD176C
:101BE0008A07D6979C43829769B905060586B73759
:101BF0000020BE95860511CA1C31A2071821D98F75
:101C00009EA1910509057D1665FA82800506058667
:101C1000B7370020BE95860519C69C411EA109054F
:101C20007D1691057DFA8280619942054181B767F1
:101C3000004023A8A7C482800A05B76700409387A5
:101C400007C03E951C4165771307F798F98FDD8D26
:101C5000C205C1810CC182800A05B7670040938725
:101C600007C03E951841E5779387F7FB7D8F4207C4
:101C7000418393F7050199C31347070193F70502C1
:101C800099C313470702E177938707085D8F4207DF
:101C9000418318C11C4193F707036388B70018C13B
:101CA0001C4193F70703E39CB7FE82800A05B767E0
:101CB0000040938707C03E951841F1779387F7F866
:101CC0007D8F420741839397350163D40700856771
:101CD0003D8F9397250163D4070089673D8FE17796
:101CE000938707085D8F4207418318C11C418D66A9
:101CF000F58F638BB700C166FD160D6618C11C41D8
:101D0000F58FF18FE39CB7FE82800A05B76700402C
:101D1000938707C03E951841E5779387F7FB7D8F42
:101D20004207418313470703E177938707085D8FD5
:101D30004207418318C11C4193F707039306000330
:101D40006388D70018C11C4193F70703E39CD7FEB3
:101D500082800A05B7670040938707C03E95184107
:101D6000F1779387F7F87D8F420741838D673D8F29
:101D7000E177938707085D8F4207418318C11C41B3
:101D80008D66F58F638AD70041667D1618C11C41A8
:101D9000F18FF58FE39CD7FE82800A05B76700407C
:101DA000938707C03E951C4113971701635E070098
:101DB0001C41C207C18305671307F7F0F98F31672C
:101DC00013070708D98F1CC182800A05B767004036
:101DD000938707C03E951C4193F7070489CF1C41A8
:101DE000C207C18305671307F7F0F98F216713074F
:101DF000070CD98F1CC18280B767004083A707C535
:101E0000C207C1830E053E95B73700203E950605F3
:101E1000858186050CC18280B767004083A707C50E
:101E2000C207C1830E053E95B737002091073E9546
:101E30000605858186050CC18280B767004083A7AF
:101E400007C5C207C1830E053E95B73700203E95F2
:101E500006050A218280B767004083A707C5C2072D
:101E6000C1830E053E95B737002091073E950605C4
:101E70000A218280B767004083A707C5C207C183D4
:101E80000E053E95B737002089073E9506050CC123
:101E90008280B767004083A707C5C207C1830E05CC
:101EA000AA97373500201905AA9786071307E0037C
:101EB000637EB70013D75500FD8981E57D17420782
:101EC00041832A07A166558F98C3828013D71500D6
:101ED0008589B335B0002E972A0798C38280B767EB
:101EE000004083A707C5C207C1830E053E95B737DB
:101EF000002099073E95060508411375F53F82803D
:101F0000935785001375F50F22055D8D8280376725
:101F10000040232207C4F177938707F02392F18AC8
:101F2000B167938707F02320F7C401458280EFE271
:101F30002FA42E8932849374F5072685FD3D420433
:101F400041802286AA854A85EFF03FCAA285268570
:101F5000153701456FE00FA4EFE28FA12E8993742E
:101F6000F5072685AD3F2A842685F5352286AA8584
:101F70004A85EFF0BFC922856FE0CFA101A001A083
:101F800001A001A001A001A001A001A001A001A049
:101F900001A001A001A001A001A001A001A001A039
:101FA00001A001A001A001A001A001A001A001A029
:101FB00001A001A001A001A001A001A001A001A019
:101FC00001A001A001A001A001A001A001A001A009
:101FD00001A001A001A001A001A001A001A001A0F9
:101FE00001A001A001A001A097F1FF1F9381819C96
:101FF000171100201301018117450000130505E2A8
:1020000097E5FF1F938505001386818563FAC50058
:102010008322050023A0550011059105E3EAC5FEC2
:10202000138581859385816A6377B5002320050038
:102030001105E36DB5FEFD42739002BC8D427390B5
:1020400042809302800873A0023097E2FFFF9382E0
:10205000E2FE93E2320073905230EF00400197129B
:1020600000009382228C7390123473002030B717D3
:10207000024098431367170098C3D843B706FFF888
:10208000758FD8C39843B706F7FEFD16758F98C3B2
:102090009843B706FCFFFD16758F98C3D843B70663
:1020A00081FFFD16758FD8C337079F0098C7B746C5
:1020B000024003A706801367070123A0E680D843E8
:1020C000D8C3D843D8C3D84313670740D8C3D8432D
:1020D000B706C1FFFD16758FD8C3D843B7063C00BD
:1020E000558FD8C39843B7060001558F98C39843BE
:1020F00093166700E3DD06FEB7170240D843719BD5
:10210000D8C3D84313672700D8C3B7160240214766
:10211000DC42B18BE39EE7FE82801C4161773D0784
:102120007D8F9C459451D58F9449D58FD449D58FB7
:10213000944DD58FD44DD58FD451D58F9455D58FFF
:10214000D98F1CC1DC455CC19C411CC5DC415CC510
:10215000828091C51C4193E717001CC182801C41FD
:1021600041677917F98F1CC182804CC18280484138
:102170004205418182805C45D9C3B70601409387FF
:10218000064003A6064018411347F7FF718F23A0AE
:10219000E64083A6464018411347F7FF758FD8C322
:1021A00058413E9714431041D18E14C394471841AF
:1021B0001347F7FF758F98C7D44718411347F7FFA8
:1021C000758FD8C71C454147638CE700370701402E
:1021D00013070740BA9798431441558F98C38280DC
:1021E000B707014003A787401441558F23A4E74058
:1021F00003A7C7401441558F23A6E740828058416A
:10220000B7070140938707403E9714431C4193C78B
:10221000F7FFF58F1CC38280B707014023AAA740B0
:1022200082809C4593F8F700C18B81C7DC41B3E8FD
:10223000F800B7270240985BB707000FF98F89EFC6
:1022400005472385E18AB7170140631BF5009E21EE
:10225000B5839EA181EB8280B7170140630EF50024
:102260009C21A1CF10418147054E3D4F930E800226
:10227000930F8004214309A883C7A18AF5D3C1BF66
:1022800054C98507638A6702B316FE009A21758FC9
:10229000E399E6FE139727003318EF001348F8FF81
:1022A0003376C8003397E800598E9845E30AD7FD86
:1022B000E319F7FD14C9F1B710C19A219307F00F84
:1022C00063FCE7045041A147054EBD4F130F800248
:1022D000930E8004414331A054C90DA88507638C37
:1022E0006702B316FE009A21758FE399E6FE1397F5
:1022F000270001173398EF001348F8FF3376C80022
:102300003397E800598E9845E308E7FD9845E317B1
:10231000D7FD14C9E1B750C18280B71701406304EB
:10232000F5000CC9828083C7A18AE5DFB581D5BFDE
:1023300083A7C18A85EF14213C21920793F7F70FF9
:1023400037E700E036972300F7405C4163820712CD
:102350001821935757008546B396E60093870704E4
:102360008A0737E700E0BA9794C3828003A7C18A3F
:102370008547630CF70203A7C18A89476302F70602
:1023800003A7C18A8D476301F70A03A7C18A914752
:10239000E31DF7FA14211C31920793F7F70F37E783
:1023A00000E036972300F7404DB71831630DF70072
:1023B00014213C21920793F7F70F37E700E0369797
:1023C0002300F74059B714213C21920793E707F8FF
:1023D00093F7F70F37E700E036972300F740B5B7DC
:1023E0001C3105476375F70214219387E7038A07B9
:1023F0003821BA9793F7F70F920793E707F893F707
:10240000F70F37E700E036972300F7403DBF142170
:102410008A073821BA97920793F7F70F37E700E05A
:1024200036972300F74015B71C310D47636FF7004F
:10243000142186073821BA97920793F7F70F37E7E9
:1024400000E036972300F74009B714219387C707A8
:1024500086073821BA9793F7F70F920793E707F8A3
:1024600093F7F70F37E700E036972300F740F1BD09
:102470001821935757008546B396E60093870706C1
:102480008A0737E700E0BA9794C38280B717024003
:10249000D843B70640FFFD16758FD8C3D8435A05F9
:1024A000598DC8C38280B7170240DC43B18B1147F6
:1024B000638EE70621476381E70899C7B7177A005B
:1024C000938707201CC131A0B7177A009387072094
:1024D0001CC1371602405C429183BD8B3707002038
:1024E0001307C719BA9794231C41B3D7D7005CC10F
:1024F0005442A1829D8ABA969422B3D6D70014C5BD
:102500005442AD829D8A36971823B3D7E7005CC545
:1025100058423983937637001387018436971823FE
:102520001377F70FB3D7E7021CC98280B7177A0079
:10253000938707201CC171BF371702405C43584383
:10254000C166758FC983BD8B8907C5466381D70274
:102550000DEB3747024003270780418B19CB371714
:102560007A0013070720B387E7021CC19DB7C9474C
:10257000C5B737173D0013070790B387E7021CC1A3
:1025800089BF3717024058439316E70063DA060005
:1025900037173D0013070790B387E7021CC115BF2B
:1025A00037177A0013070720B387E7021CC115B756
:1025B00099C5371702405C4B5D8D48CB8280B717B9
:1025C0000240D84B1345F5FF798DC8CB828099C561
:1025D000371702401C4F5D8D08CF8280B71702402D
:1025E000984F1345F5FF798D88CF828099C53717AD
:1025F00002405C4F5D8D48CF8280B7170240D84FB4
:102600001345F5FF798DC8CF8280EFD27FB60111D7
:102610002A84AE841A29F577FD17F98FFA21D98F0C
:102620001EA95A25FD779387379FF98FDA21D98F15
:102630009A25D98FBA25D98F5EA55E29C207C18395
:1026400093F7F7CFDA25D98F5EA96800EFF0BFE5E1
:10265000B747014093870780630CF40452475E2418
:10266000C207C18763C8070493171700BA978E077C
:10267000BA9798400A07B3D7E70213074006B3D6C4
:10268000E7029206B3F7E7025A2442074187634DF7
:10269000070292079387270313074006B3D7E70281
:1026A000BD8BD58FC207C1831EA405616FD09FAEBD
:1026B000624775B793171700BA978E07BA97984075
:1026C0000607B3D7E70255BF139737001307270351
:1026D000930740063357F7021D8BB367D700D9B76E
:1026E00091C55E250967D98F5EA582805A25F97745
:1026F000FD17F98F5EA5828009C65E29DD8D4EA982
:1027000082805E2993C5F5FFFD8D4EA98280B7F7C3
:1027100000E023A0070023A207008146014794C7D9
:10272000D8C7814688CBD4CB3D4798C3B7E700E0F4
:10273000056723A0E7108280B7F700E023A2070017
:102740009387018B9843050798C373002030EFD01F
:10275000BFB57300203037050400EFF0FFAB730006
:102760002030EFD2FFA0AA842E8485451145EFF0DA
:102770001FE6B1CCB766004083A706C44167751752
:10278000F98F23A0F6C4B717014003A74780B716F7
:10279000F0FFFD16758F23A2E78003A7C780F976A7
:1027A0009386F67F758F23A6E78003A74780B746F9
:1027B0000400558F23A2E78039CC37470240832796
:1027C000078093E727002320F7806FD0BF9C3767EF
:1027D0000040832707C493E72700C207C183232053
:1027E000F7C4B717014003A74780B716F0FFFD16DF
:1027F000758F23A2E78003A7C780F9769386F67FBB
:10280000758F23A6E78003A74780B7360300558F4F
:1028100023A2E78055B73747024083270780F59BFF
:102820002320F7805DB783A7C1830567130707FAE5
:10283000B3D7E702B387A70299CF0147856693868E
:1028400006FA0100050783A7C183B3D7D702B38770
:10285000A702E368F7FE82801DC6AE870606B29522
:10286000A54611A81307770398A3A38007001205B4
:102870008907638AB7001357C501E3E5E6FE13072E
:10288000070398A3DDB78280EFD29F8E011109451F
:10289000EFF0DFBF854537058000EFF03FD5B7F794
:1028A000FF1F83A4C77E03A4077F03A5877E21465D
:1028B000B70500209385E50C2295793F1146B705B1
:1028C00000209385E50D338584007937EFE03FE6FE
:1028D00093074002230CF1008547A30CF100230D60
:1028E0000100054422CE2808EFF09FA4370504001C
:1028F000EFF09F92B70704003EC402C6C1473EC82E
:1029000022CA2800EFF03F879307A003230CF100B1
:10291000A30C01002808EFF0BFA105616FD09F87CD
:10292000EFD21F85EF10207A3128B93F03A5C1836C
:102930009307803E3355F502EFF07FDDEFD01FB6F1
:102940007D2AEDBFEFD23F815D7185451145EFF0E6
:102950001FC8854537050200EFF05FC9854505456D
:10296000EFF01FC591472312F104E147BEC68D4722
:10297000BEC4CC003714014013050480EFF07F8AF9
:10298000A1472312F10493078004BEC6CC001305AF
:102990000480EFF01F89C1473EC837440040130A46
:1029A000444052C402CC9387C1D83EC613090008E4
:1029B0004ACE02D002D202CA89694ED602D402D8C7
:1029C0002C00B704024013850408EFF00FF585458D
:1029D00013850408EFF0EFF702C852C402CC9387C6
:1029E000C1D03EC64ACE02D002D24ACA4ED69307C2
:1029F00000023ED402D82C001385C406EFF0EFF19C
:102A000085451385C406EFF0CFF4F167938707205F
:102A10003EDA231C0102231D0102231E0102B147DD
:102A2000231FF102231001044C1813050440EFF09A
:102A3000DFBD05469305000C13050440EFF0DFCB26
:102A4000854513050440EFF0BFC961616FD0EFF316
:102A5000EFD20FF24111231201005C310547638C64
:102A6000E70213978701618719C70947638BE7025C
:102A70002314010019A0231401005C210547638A77
:102A8000E7061397870161871DC309476386E70639
:102A90002313010039A8930700607C8485677C823A
:102AA000E9BF930700407C8485677C82F9B72313D4
:102AB00001001C21183122075D8F3C21C2075D8F68
:102AC0003C31E207D98F3EC0B1477C852316010017
:102AD0001964731004808A8537450040130505404A
:102AE000EFF0BFB2130484087310048041016FD06B
:102AF0006FEA8D677C8375BF89677C835DBFEFD28A
:102B00002FE7B70700201387C7778567BA9783D762
:102B10000785C207C18399EFB70700201387C777DE
:102B20008567BA9783D74789C207C1836391070E28
:102B30006FD04FE6370502401305C506EFF02FE3CF
:102B400013040008098C83A7818BB306F440130794
:102B5000F003636FD700638C870683A6018B03A7FE
:102B6000418B6386E6066371F4021304000829A012
:102B70006374F400130400083307F4409306000460
:102B800063F4E60013840704B306F440C206C1826E
:102B9000370700201306C777056732972317D784B6
:102BA000231807840356E7849385C1D0BE95130587
:102BB0003008EFF0CFB70D45EFF02F951374F40701
:102BC00023AC818A03A7018B23AAE18AB1B7B70797
:102BD00000201387C7778567BA9783D7E784C20732
:102BE000C18313070004E399E7F2B70700201387B6
:102BF000C7778567BA9723970784014681451305F0
:102C00003008EFF0CFB20D45EFF02F9031B7370518
:102C1000024013050508EFF08FD5E31B05F03704DC
:102C200000209307C47705643E94231A0488035652
:102C300024899385E1611385C1D8EF20107A8145FD
:102C4000B704024013850408EFF0AFD08355248900
:102C500013850408EFF06FD1854513850408EFF064
:102C60004FCF0D45EFF0EF8EE1B5EFD26FCD79711B
:102C70002A892E841C2193C607087D476371D702D9
:102C8000938C15009CA175476374F7006F10803416
:102C90008A071967130787D9BA979C438287EF1071
:102CA000805149AC1C311307000F6389E708637733
:102CB000F7021307E00F6381E70A6368F708130759
:102CC000100F01456396E706238105008557BCB1C7
:102CD000D557DCA19547DCB1114599A81147638A06
:102CE000E702254701456395E70413872500B76789
:102CF000000003C807E1938707E18833AC23B033B2
:102D0000D4232301040108B32CA330B354A31545E5
:102D100005A09387018588238C33B023B433D8234F
:102D2000DC3328A02CB050A054B078A07CB019455A
:102D300008B0B707020089073E95EDAA9307300354
:102D4000BCA1A38105000945E5B793070004BCA118
:102D5000A38105000945E9BFA147BCA10545C9BF3D
:102D60001C3191CB0547638EE702FD579CB13705B7
:102D7000020005056DAA3C21858B89CFB71701405C
:102D80001307000223A8E780A30004003705020010
:102D9000050571AAB71701401307000223AAE780AF
:102DA000E5B73C21858B81CBB717014013070002A3
:102DB00023A8E780D1BFB71701401307000223AA59
:102DC000E780D9B71C3189CB05476387E7000947FE
:102DD000638CE7048147A9A005472382E166894502
:102DE000B714014013850480EFF02FD38545138578
:102DF0000480EFF08FD289472312F102C1473ED6FB
:102E00008D473ED44C1013850480EFF08FC1854769
:102E10002312F1024C1013850480EFF08FC0854718
:102E20001CB04165050521A209472382E166894559
:102E3000B714014013850480EFF02FCE854513852C
:102E40000480EFF08FCD9305000813850480EFF028
:102E5000CFCC89472312F102C1473ED68D473ED4DD
:102E60004C1013850480EFF0CFBB85472312F1028D
:102E70004C1013850480EFF0CFBA9307000823129B
:102E8000F1024C1013850480EFF0AFB993070004F2
:102E90002312F102930780043ED64C101385048060
:102EA000EFF02FB88947ADBF2382016685451145F4
:102EB000EFF0EFF185452145EFF06FF189492312DD
:102EC000310391473ED68D473ED44C10B714014094
:102ED00013850480EFF0EFB40549231221034C1051
:102EE00013850480EFF0EFB3231231034C101385E8
:102EF0000480EFF00FB3231221034C1013850480DC
:102F0000EFF02FB2930700082312F1024C10138543
:102F10000480EFF00FB1930700042312F1024C106C
:102F200013850480EFF0EFAFA30004000545C164F2
:102F30008504269545616FD06FA43C21A207183106
:102F40005D8F93171700BA979207FD17FDFFA30037
:102F50000400370502000505D9BF23810500A380C1
:102F600005000945E9B71431368503472900834731
:102F70004900A207034659004206D18F0346390093
:102F8000D18F034669006206D18F1376170009CAF4
:102F900093F51600E5C5B7150140094823A805813A
:102FA00013782700630A080093F52600F1CDB715C2
:102FB0000140854823A8158193784700638C080059
:102FC00093D526008589F9C5B7150140130300087C
:102FD00023A8658013138701135383416343030CB4
:102FE000A9CF13DE160093DE260013DF56009D8264
:102FF000B71501401377070219C683A7858085831B
:10300000858BE31BF5FE6307080083A78580858B0E
:10301000E314FEFE6388080083A785809D83858B6B
:10302000E39CFEFC19C3E3190FFC6358030083A75C
:1030300085809183858BE391F6FC37170140032649
:10304000878083278780832587808326878013074F
:1030500007801847858B860795819189CD8F0582DA
:10306000058AD18F8D82A18AD58F0E071377070825
:10307000D98F1CB037050600050555BDB7150140B1
:10308000094823AA058129BFB7150140854823AA0D
:1030900015811DB7B71501401303000823AA6580E9
:1030A00015BF93D5760099C5B7150140414E23A8A9
:1030B000C5813DB7B7150140414E23AAC5810DB763
:1030C0003C21A20738314207D98F1831D98F5821B6
:1030D0006207D98F9DC3375725021307F70F637413
:1030E000F70293874166054798B30547D8C3A30005
:1030F00004003705040005051DBDFD579CB13705CB
:10310000040005052DB5A382016637A74A041307FD
:10311000F71F3E97B357F7028946054763F5F60058
:103120000D4733D7E70223A4E166D1B79305250005
:10313000043199E0930400102685EF204004A30099
:103140000400138574000D81050542051365150003
:10315000F9BB1C311387416693F63700850614AF1F
:103160008983858B1CBFA380050041650505C1B31C
:10317000938A2500A38005009307250003491500C5
:10318000854C0544FD5B130C0004B7190140054B49
:103190001DA823A8698183A70980C19B93E78700A5
:1031A00023A0F9805686D285EF20E002631409003F
:1031B0006F0010700504A69AA69CD28729A0B307B9
:1031C0009A00050426947D19630A7905138A17006D
:1031D00088239377F50391E3E2879D0793D4370023
:1031E00093178501E187E3C607FA23AA698183A7BC
:1031F0000980C19B93E7370023A0F9805686D285CA
:10320000EF10707DE31D09FA23AA698183A7098065
:10321000C19B93E7370023A0F98055B7131504012C
:103220003365950129B3138A2500A3800500930710
:10323000250083491500854C0544FD5A130B0004F5
:1032400015A09D048D805286DE854A85EF0050775B
:10325000B3879B00138714003A946209135989417C
:10326000634E0900FD19638E5901938B170003C942
:1032700007009374F903F1F4DA84E1B7269AA69C67
:10328000D5B7131504013365950155B11306250013
:103290001C31238FF166A9C313854166710593869E
:1032A0004166138727003A999385416601470506D1
:1032B0000348F6FF23000501DAB1429705058905A9
:1032C000E31726FF3385D7003686CC2E0D8F5ABAEA
:1032D00085060906E39BA6FEA300040013851700DC
:1032E000420513651500A1B103C7416689476319FB
:1032F000F700183193874166B8BFBC2F6367F700AA
:10330000FD571CB0416505051DB13945EF1000366C
:10331000EF007079A300040028A0935785003CB00B
:10332000935705015CA0618148B04165150501B165
:10333000183193874166D8A7383122073421558F39
:103340009AAB583122075421558FBAABA3800500A0
:10335000370505000505E1BE930715003ECE03C7FE
:1033600041663AC885476305F70289476307F74610
:10337000930735003421E3970606A30004002301D8
:10338000040072473385E74042051365250045B6C2
:10339000138D3500238E018A130A3500034C250056
:1033A000630A0C4202CC014502C6014B938A416676
:1033B00089493E8985AC4C102245EF10106F631E81
:1033C0003501E3870B429387C18B9C2393F7F70F5B
:1033D000FD1BF5D36F00D041014B8547E310F54C41
:1033E00092572300FD0013D78700A300ED0013D7E9
:1033F00007012301ED0013074D00E183A301FD0048
:10340000630C0B0293978401E18763C507005A851B
:103410003A8D25A083A78A002302FD0013D78700D9
:10342000A302ED0013D707012303ED00E183A303FB
:10343000FD005A85210D11A03A8D93F70401C5CBEB
:10344000834B2A00A20B83473A00C207B3EBFB0071
:1034500083471A00B3EBFB0083474A00E207B3EB54
:10346000FB0093075A003ECA03DA2A0185889DC4EF
:1034700083D40A0181452245EF103063631D350175
:10348000E38E04409387C18B9C2393F7F70FFD14C1
:10349000F5D36F00B0408547E312F540854D1DA080
:1034A000E313B54183A74A011257F98F6385FB26C1
:1034B000E3010A3E9387C18B9C2393F7F70F7D1A94
:1034C000E399073C83D40A014C102245EF10F05DCC
:1034D000E31835FDE387043A9387C18B9C2393F768
:1034E000F70FFD14F5D389473EC86F00D03903DAD2
:1034F0000A0193F71400B5C763050B00524A02CCCA
:1035000029A281452245EF10505A631D3501E30978
:103510000A2C9387C18B9C2393F7F70F7D1AF5D361
:103520006F00D0378547E31BF536E204E18463C6BC
:1035300004005ACC2A8B524AC9A883A78A002300C8
:10354000FD0013D78700A300ED0013D70701230167
:10355000ED00E183A301FD005ACC2A8B110D524AE4
:103560006DA04C102245EF105054631D3501E30748
:103570000A329387C18B9C2393F7F70F7D1AF5D3FB
:103580006F00D0318547E31BF530E204E18463C46A
:10359000040292572300FD0013D78700A300ED001B
:1035A00013D707012301ED00E183A301FD00110DF5
:1035B000524A02CC99A883A78A002300FD0013D7A2
:1035C0008700A300ED0013D707012301ED00E1837D
:1035D000A301FD00110D75BF631A0B0883472A0074
:1035E000A20703473A004207D98F03471A00D98F31
:1035F00003474A006207D98F3ED2150A13F7040227
:1036000045CF23AAFA00014B0545B24785073EC6C0
:103610009387C18B9C2393F7F70F639007127D1C50
:10362000630F0C1093071A003ECA83440A0026C495
:1036300093F72400D5D3E3020BE083DB0A0193F771
:1036400014010547E389E7D64C103945EF10F045E2
:10365000E31435D9E38D0B189387C18B9C2393F723
:10366000F70FFD1BF5D3014B6F00901883DB0A01A8
:103670004C103945EF107043631D3501E3800B2278
:103680009387C18B9C2393F7F70FFD1BF5D36F0036
:10369000F0208547E314F52092572300FD0013D74F
:1036A0008700A300ED0013D707012301ED00E1839C
:1036B000A301FD00110D1DB703DB0A014C102245CB
:1036C000EF10B03E631F3501E30E0B109387C18BE3
:1036D0009C2393F7F70F7D1BF5D352CA014B6F0064
:1036E000F01B8547E312F510E204E1842ACC014B7C
:1036F000E3DD04F083A78A002300FD0013D78700D1
:10370000A300ED0013D707012301ED00E183A3011E
:10371000FD00110DDDBD524A02CCC5BD150A11A038
:10372000150A7D1C630D0C0083470A0013F7270060
:1037300065DBC18BE5F7050AEDB7E3170CFE85479E
:10374000630FF500B2471CB028A0F2473305FA40DA
:103750004205B30C9D41336595016FF04FFD630742
:103760000B0483D4416709494C103945EF10F033FD
:10377000631B2501E1D89387C18B9C2393F7F70F37
:10378000FD14FDD3C1B78547E31EF5FA9257230018
:10379000FD0013D78700A300ED0013D70701230115
:1037A000ED00E183A301FD00110D69BFE247D9DB04
:1037B00083D44167094981453945EF10102FE31340
:1037C00025F9C9D09387C18B9C2393F7F70FFD147C
:1037D000FDD38DBF62C66285B5B7938D3500238E4C
:1037E000018A183193874166B8BFBC2F637EF73CCE
:1037F00093043500834B2500638D0B3C02C602CA3F
:10380000014A138D41668949D9AAA94752476316CF
:10381000F7024C103945EF10202163143503E38B78
:103820000A049387C18B9C2393F7F70FFD1AF5D3F6
:10383000A9473ECA814A6F0030042945EF00106352
:10384000C9BFA9473ECA014A85476315F57A925711
:103850002380FD0013D78700A380ED0013D7070155
:103860002381ED0013874D00E183A381FD006302F6
:103870000A7A93178B01E18763C90700BA8D137B1E
:103880000B01631E0B78E24435AA83278D00238247
:10389000FD0013D78700A382ED0013D70701238310
:1038A000ED00E183A383FD00A10DD1BF6285EF0090
:1038B000F05B6F00807985476305F502B1A8054785
:1038C0006315E57E83274D011257F98F6307FB22AD
:1038D000638C0A049387C18B9C2393F7F70FFD1A1F
:1038E000A9E383540D014C102245EF10E013E318B7
:1038F00035FD81C89387C18B9C2393F7F70FFD1487
:10390000FDD383A781671257F98F63876701C24789
:1039100013E507011375F50F62CAE24463980B1EA5
:103920002DAC85473EC8E5B785473EC8CDB7D247E1
:103930006396870383540D0181452245EF10C00E25
:103940002A8A631135036389046A9387C18B9C2398
:1039500093F7F70FFD14EDD3014A7DBF6285EF00A9
:10396000F050C9BF8547631BF568620B135B8B4141
:1039700062CAE246B68463570B0483278D00238016
:10398000FD0013D78700A380ED0013D70701238123
:10399000ED00E183A381FD00910D2DA063190A08BC
:1039A000BC20A207B8304207D98F9830D98FD820D1
:1039B0006207D98F3ED2950413770B0269CB232A75
:1039C000FD00014AB24785073EC69387C18B9C2301
:1039D00093F7F70F63940714FD1B63840B1493870D
:1039E00014003ECC03CB04005AC4137C1B00290CEA
:1039F00093772B00C5D7630F0A60835A0D01D24716
:103A0000E39587E193770B01E39107E04C102245A2
:103A1000EF108001E31A35E3638C0A649387C18B4E
:103A20009C2393F7F70FFD1AF5D3D28AB1A5A947C6
:103A300052476315F702835A0D014C103945EF00C8
:103A4000B07E63113503638D0A5A9387C18B9C2323
:103A500093F7F70FFD1AF5D3294C7DBD2945EF00EB
:103A6000F040D1BF8547631FF55892572380FD0072
:103A700013D78700A380ED0013D707012381ED0042
:103A8000E183A381FD00910DA9473ECA11BFD24732
:103A90006316FC02035A0D014C102245EF00D0784A
:103AA0006312350363020A569387C18B9C2393F7F5
:103AB000F70F7D1AF5D326CC014AB9BD6285EF0018
:103AC000F03AC9BF85476313F554620B135B8B4112
:103AD00062CA014AE3580BEE83278D002380FD0064
:103AE00013D78700A380ED0013D707012381ED00D2
:103AF000E183A381FD00910DF1B562CAE244D9B51D
:103B0000950411A09504FD1B63860B049C2013F7FC
:103B100027006DDBC18BEDF78504F5B70545E3970D
:103B20000BFEA94752476317F704630C0A0603D933
:103B3000416789494C103945EF00106F6310350516
:103B4000630D09009387C18B9C2393F7F70F7D19B1
:103B5000F5D321A08547E306F5FCB2471CB028A0A9
:103B6000F2473385F4404205B38C9D41336595019E
:103B70006FF0EFBB2945EF00702F45BF8547E31E6F
:103B8000F5FC92572380FD0013D78700A380ED003A
:103B900013D707012381ED00E183A381FD00910D7F
:103BA0006DBF03D94167894981453945EF00D06729
:103BB000E31535FBE30309FA9387C18B9C2393F745
:103BC000F70F7D19F5D351BF93042500014502C6B7
:103BD00069B75E855EC651B7950711A09507FD16BA
:103BE000638D06F89823137627006DDA418B6DF705
:103BF0008507F5B783C741660547638DE700094729
:103C0000638CE716A380050023810500A3810500CE
:103C10000D454DAC93844500238E018A034C35003D
:103C2000220C3C21336CFC00630F0C125C213E8A99
:103C300013F7270001EB130D5500814B938D41665F
:103C4000894A5DA0858B85CB83DB416789498145A6
:103C50005285EF108065631D350163880B0C9387D7
:103C6000C18B9C2393F7F70FFD1BF5D3814B75A8F0
:103C70008547631DF50E7D1C814B138D4166894A76
:103C8000854D0DA893771A0085CB394A35A0631E60
:103C9000B50992579CA013D7870098B013D7070196
:103CA000B8A09104E183A38FF4FE850B7D1CFD5722
:103CB000630DFC06E3080CFC83590D014C10528582
:103CC000EF10A05EE31555FD638109069387C18B54
:103CD0009C2393F7F70FFD19F5D381A88547631649
:103CE000F504850B630D7C0583471D00A207034780
:103CF0002D004207D98F03470D00D98F03473D00A0
:103D00006207D98F3ED2110D83D90D014C10528517
:103D1000EF10A059E31455FD638909009387C18B07
:103D20009C2393F7F70FFD19F5D3A300740193DBE0
:103D30008B002301740128B03385944161A283D99B
:103D40004167094A81453945EF1020566312450302
:103D5000638209029387C18B9C2393F7F70FFD19A8
:103D6000F5D3E28BD9B76285E28BC1B7814B75BFC2
:103D7000E28B65BFE28B55BF93844500238E018A99
:103D8000183193874166B8BFBC2F6372F718034D93
:103D90003500220D3C21336DFD00630D0D16834966
:103DA00045004E8A93F71900A9073EC43E85EF00EF
:103DB000F00B93F9290063990900130C5900014B8A
:103DC000938D4166894A6DA003DB4167894981452E
:103DD0005285EF007045631D3501630C0B0C938712
:103DE000C18B9C2393F7F70F7D1BF5D3014BD1A01B
:103DF00085476314F5127D1D014B138C4166894A7A
:103E0000854D2DA8394AA2472947638BE7022945EA
:103E1000EF00D00535A0631EB50992579CA013D7BB
:103E2000870098B013D70701B8A09104E183A38F4E
:103E3000F4FE050B7D1DFD57630DFD06E3040DFC2F
:103E400083590C014C105285EF00103EE31555FDCF
:103E5000638109069387C18B9C2393F7F70FFD19A4
:103E6000F5D381A885476316F504050B63056D0737
:103E700083471C00A20703472C004207D98F034742
:103E80000C00D98F03473C006207D98F3ED2110C3A
:103E900083D90D014C105285EF001039E31455FD04
:103EA000638909009387C18B9C2393F7F70FFD1952
:103EB000F5D3A3006401135B8B002301640128B0D8
:103EC0003385944183474900898BB1CFB7040400FF
:103ED000458D6FF0CF85A94722476316F70283D936
:103EE0004167094A81453945EF001034631945039C
:103EF000638909029387C18B9C2393F7F70FFD1900
:103F0000F5D36A8B7DB72945EF004076C9BF0145DF
:103F1000014B45B76A856A8B69BF014B59BF6A8BF4
:103F200049BF6A8B79B783443900A20483472900CB
:103F3000DD8C8504CA04458D6FE07FFF83C7416631
:103F40000547638CE7000947638FE702FD579CB183
:103F50003705050005056FE09FFD3C31A20758219C
:103F60004207D98F3821D98F58316207D98F3ED275
:103F70004C100145EF106033A30004003705050025
:103F800005056FE0DFFA183193874166B8BFBC2F93
:103F90006369F700FD579CB13705050005056FE023
:103FA0001FF92145EF00806C83473900A2070347C2
:103FB00049004207D98F03472900D98F034559008B
:103FC00062055D8D0529A300040037050500050580
:103FD0006FE0FFF5FD571CA0416505056FE09FF5FB
:103FE000528B6DA852CA5DA852CA014B45A85E8B80
:103FF00009456DA0524C0DB2268A39BA014A29BA38
:10400000294C19BA294C09BA26CC39B226CC014A16
:1040100021B2BA8D93770B01014AE38A079003CB53
:104020002400220BBC30C207336BFB009C30336B87
:10403000FB00DC20E207336BFB00938754003ECC8F
:10404000835A2D01D247E313FC8683540D01814529
:104050002245EF00701DE3103587E38F048A9387B4
:10406000C18B9C2393F7F70FFD14F5D36FF0DF8A14
:10407000D28A19A0A9473ECA524C568A09456FF008
:10408000BF8989473EC883A781671257F98F638725
:10409000FB00C24713E507011375F50F524A63157C
:1040A0000CE86FF02FEA2AC8F9BF2AC86FF07F85A5
:1040B00023AA698183A70980C19B93E7370023A0C6
:1040C000F9806FF02F8FEFC20F89411193874166FE
:1040D00023800700A3800700C144C4C323860700D0
:1040E000130740069AAB2399070023AA0700054748
:1040F00098AFA38C0700238D070085451145EFE09D
:104100000FCD85452145EFE08FCC094A23124101AF
:1041100091473EC68D494EC44C00371401401305EB
:104120000480EFE00F900549231221014C00130594
:104130000480EFE00F8F231241014C00130504802F
:10414000EFE02F8E231221014C0013050480EFE0D5
:104150004F8D930700087C824C0013050480EFE02C
:104160004F8C930700047C824C0013050480EFE021
:104170004F8B130900022312210126C64EC44C00A6
:1041800013050480EFE0EF89231221014C00130591
:104190000480EFE00F89C14513050480EFE0EF973D
:1041A0006482D1473EC64C0013050480EFE06F8760
:1041B00041016FB09FFD1C219CA1416505058280D6
:1041C0001373F503631403001303000493770504CA
:1041D0008DCFB7170140054723A8E7806304030C80
:1041E000411122C626C44AC24EC0937305088149B4
:1041F000A1441384416637180140130808809302D4
:104200000008094FFA8F1D4995A0B71701400547CF
:1042100023AAE780E1B7232A5800232AF801F2876E
:10422000FD17FDFF83278800998313F717002328C4
:10423000E801F287FD17FDFF93D818000581931759
:1042400077005D8DB307D300FD166389D6019DCE3F
:1042500093F71800E9D323285800C1B77683638504
:10426000030008A27683050663080302850583C858
:10427000F5FF630B0300032E4400930E83FF9A8621
:10428000014533036940E9B71A85A68763860300B1
:104290003355F500CE8EF1B73244A244124982491B
:1042A000410182808280B7170140054723A8E7803B
:1042B000094723AAE78083A68166B687FD17FDFF1D
:1042C000B7170140094723A8E780B687FD17FDFF10
:1042D000B7170140054723AAE780094723AAE780CB
:1042E000B687FD17FDFFB7170140094723A8E780F0
:1042F000B687FD17FDFFB7170140094723AAE780DE
:10430000B687FD17FDFFB7170140094723A8E780CF
:1043100036857D157DFD83C7F16795C3371601404E
:104320001306068089452E88232A060136877D17C5
:104330007DFF0CCA36877D177DFFFD17F5F7FD451C
:1043400037160140130606800948C288232A160141
:10435000B687FD17FDFF18469357670013F7170040
:1043600023280601B687FD17FDFF9317F701C98FB4
:1043700013D51700FD15F9F9B7170140054723A814
:10438000E780094723AAE780B687FD17FDFF3716A8
:10439000014083278680998313F7170089472328D4
:1043A000F680B687FD17FDFF9317F7015D8DB717F0
:1043B0000140094723AAE780B687FD17FDFFB7171D
:1043C0000140094723A8E780B687FD17FDFFB7170F
:1043D0000140054723AAE780094723AAE780B6875B
:1043E000FD17FDFFB7170140094723A8E780FD1619
:1043F000FDFE8280B7170140054723A8E7800947E3
:1044000023AAE78003A68166B287FD17FDFFB717D1
:104410000140094723A8E780B287FD17FDFFB717C2
:104420000140054723AAE780094723AAE780B2870E
:10443000FD17FDFFB7170140094723A8E780B287A2
:10444000FD17FDFFB7170140094723AAE780B28790
:10445000FD17FDFFB7170140094723A8E780B28782
:10446000FD17FDFF03C7F16715C3B716014093861B
:10447000068089452E8823AA0601B287FD17FDFF15
:104480008CCAB287FD17FDFF7D1775F7B71701407E
:104490001307000823AAE780094723AAE780B28709
:1044A000FD17FDFFB7170140094723A8E780B28732
:1044B000FD17FDFFB7170140094723AAE780B28720
:1044C000FD17FDFFB7170140094723A8E780B28712
:1044D000FD17FDFFB7170140094723AAE780B28700
:1044E000FD17FDFFB7170140094723A8E780B287F2
:1044F000FD17FDFFFD46371701401307078093089E
:10450000000889452E8839A8232A1701232A070184
:10451000B287FD17FDFF0CCBB287FD17FDFF0581AC
:10452000FD1699C693771500E5D323281701F9BF27
:1045300093874166B42FBC3F9D8E85476382F60EFC
:10454000058961C9B71701401307000823A8E78050
:10455000B7170140094723AAE78003A78166BA87F6
:10456000FD17FDFFB7170140094623A8C780BA878A
:10457000FD17FDFFF9168DC23716014013060680A0
:1045800089452E8548CABA87FD17FDFF0CCABA8730
:10459000FD17FDFFFD16FDF6B7170140854623A860
:1045A000D780894623AAD780BA87FD17FDFFB717A2
:1045B0000140894623A8D7807D177DFFB7170140AA
:1045C000094723AAE78083A781663E877D177DFF81
:1045D0003717014089462328D7803E877D177DFF06
:1045E000371701408546232AD7808946232AD7805A
:1045F0003E877D177DFF3717014089462328D780E6
:10460000FD17FDFFB71701401307000823A8E78037
:104610008280B71701401307000823AAE7800DBF67
:10462000B7170140054723A8E78005890DC9B717CB
:1046300001401307000823A8E780B7170140094786
:1046400023AAE78083A781663E877D177DFF371702
:10465000014089462328D780FD17FDFF85B7B7178E
:1046600001401307000823AAE780C1BF83C7516632
:10467000638F0714B7170140854623A8D7800947E1
:1046800023AAE78023A8E78023AAE78023A8E7805E
:1046900023AAD78023AAE78023A8E78023AAE7805C
:1046A00023A8E7801307000823A8E78093874166C3
:1046B000B83F21070607BA97DE2B91CB3717014089
:1046C00013070780894654CB14CBFD17EDFF938762
:1046D0004166B83FBA97D82F7D1705C7B717014075
:1046E0009387078013060008894639A0D0CBD4CB26
:1046F00094CB05817D1711C793751500E5D990CB33
:10470000FDB793874166B83F41070607BA97DE2B8E
:10471000D9C3058935C937170140930600082328F6
:10472000D780371701408946232AD7802328D7808E
:10473000930600082328D780FD1791CB3717014037
:1047400013070780894654CB14CBFD17EDFFB7172D
:104750000140054723A8E780094723AAE78023A84B
:10476000E780B7170140094723AAE78023A8E7801D
:10477000854623AAD78023AAE78023A8E7801307CA
:10478000000823A8E78082803717014093060008BD
:10479000232AD78079B7B7170140054723A8E780B8
:1047A000058919CDB71701401307000823A8E78032
:1047B000B7170140094723AAE78023A8E78055B728
:1047C000B71701401307000823AAE780D5B7B7172A
:1047D0000140054723A8E780094723AAE78083A76C
:1047E00081663E877D177DFF371701408946232864
:1047F000D7803E877D177DFF371701408946232AE2
:10480000D7803E877D177DFF3717014089462328D3
:10481000D7803E877D177DFF371701408546232AC5
:10482000D7808946232AD7803E877D177DFF37179B
:10483000014089462328D7803E877D177DFF3717A3
:1048400001408946232AD7803E877D177DFF371791
:10485000014089462328D7803E877D177DFF371783
:104860000140930600082328D78013874166343F10
:10487000A106860636975A2B15C337160140130634
:10488000068089452E88232A0601BE86FD16FDFE78
:104890000CCABE86FD16FDFE7D1775F713874166AF
:1048A000343F3697542FFD168DCE3717014013072E
:1048B0000780930500080948C28839A84CCB232AF1
:1048C00017013E867D167DFE232807013E867D1654
:1048D0007DFE0581FD1691C61376150065D20CCBC1
:1048E000F9BF93874166B83F41070607BA97DA2BAD
:1048F00041CF058959C1B71701409306000823A885
:10490000D780B7170140894623AAD78083A781663D
:10491000BE86FD16FDFEB7160140094623A8C680D7
:10492000BE86FD16FDFEB71601401306000823A83B
:10493000C680938606807D1711CF368689452E85E1
:1049400048CABE86FD16FDFE0CCABE86FD16FDFEDB
:104950007D177DF73717014085462328D780894684
:10496000232AD7803E877D177DFF37170140894670
:104970002328D780FD17FDFFB1A0B717014093068C
:10498000000823AAD780B5BFB7170140054723A861
:10499000E780058959C1B71701401307000823A80C
:1049A000E780B7170140094723AAE78083A78166FC
:1049B0003E877D177DFF3717014089462328D78022
:1049C000FD17FDFFB7170140094723AAE78083A71A
:1049D00081663E877D177DFF371701408946232872
:1049E000D7803E877D177DFF371701408546232AF4
:1049F000D7808946232AD7803E877D177DFF3717CA
:104A0000014089462328D780FD17FDFFB7170140D5
:104A10001307000823A8E7808280B7170140130717
:104A2000000823AAE780B5BF83C751666389072CB6
:104A3000B7170140854623A8D780094723AAE780F6
:104A400023A8E78023AAD78023AAE78023A8E780AA
:104A500023AAE78023A8E78083C7F16791CB3717A4
:104A6000014013070780894654CB14CBFD17EDFF97
:104A700093571500858BF5C3B7170140130700083E
:104A800023A8E780371601400947232AE6808327B9
:104A900086802328E68013060680958393F62700F8
:104AA00093572500858BE9C31307000818CAB71769
:104AB0000140094623AAC78003A787801983058B75
:104AC00023A8C78093573500858BD5C7B7170140FA
:104AD0001306000823A8C780371601400948232A77
:104AE000068183278680232806811306068091830A
:104AF000918BD58F5D8F85476306F708854614CA6D
:104B0000894654CA14CAB7170140894623AAD780D8
:104B100023A8D780054623AAC78023AAD78023A825
:104B2000D7809306000823A8D7801375050819C1FC
:104B300023A6016683C601679387F6FF81CEB71669
:104B40000140938606800946FD55D0CA90CAFD17DC
:104B5000E39DB7FE1375F70F8280B7170140130767
:104B6000000823AAE78039BFB717014013070008E0
:104B700023AAE7802DBFB71701401306000823AA18
:104B8000C78099BF93772500C5C77D460148B716F2
:104B9000014093860680894823AA16019C4623A8D3
:104BA00016019983FE07B3E7070113D817007D1696
:104BB00065F693874166B42FBC3F9D8E8547638A17
:104BC000F604371601408948232A168183278680F8
:104BD0009983858B23281681F91699CA37160140C7
:104BE00013060680232A160123281601FD16FDFA56
:104BF000B7160140054623A8C680094623AAC680E9
:104C000023A8C680E38105F0FE07B3E707019CC136
:104C1000DDBDB7160140854723A8F680094623AAC3
:104C2000C68083A786809983858B23A8C680D9BF39
:104C300094417D46B7170140938707801308000809
:104C4000894501A823A80701CCCB8CCB85827D1692
:104C500001CA93F81600E39708FE23AA0701EDB7EF
:104C6000138641663C2E303E918F0546638DC70406
:104C7000858AB9C2B71601401306000823A8C6806A
:104C8000B7160140094623AAC68023A8C680F91793
:104C900089CBB716014093860680D0CA90CAFD170B
:104CA000EDFFB7170140854623A8D780894623AA80
:104CB000D78023A8D78081BDB7160140130600080E
:104CC00023AAC68075BFB7170140054623A8C78031
:104CD000858A99CEB71701409306000823A8D7808C
:104CE000B7170140894623AAD78023A8D78021BDC2
:104CF000B71701409306000823AAD780D5B7B71786
:104D00000140054723A8E780094723AAE78083A736
:104D100081663E877D177DFF37170140894623282E
:104D2000D7803E877D177DFF371701408546232AB0
:104D3000D7808946232AD7803E877D177DFF371786
:104D4000014089462328D7803E877D177DFF37178E
:104D500001408946232AD7803E877D177DFF37177C
:104D6000014089462328D7803E877D177DFF03C7F2
:104D7000F1671DC337160140130606800948C28833
:104D8000232A1601BE86FD16FDFE23280601BE86D7
:104D9000FD16FDFE7D176DF793571500858B638B10
:104DA0000716B71701401307000823A8E780B717B5
:104DB0000140094723AAE78083A781663E877D17C4
:104DC0007DFFB716014003A786801983058B09462E
:104DD00023A8C680BE86FD16FDFE131817001357C4
:104DE0002500058B630F0712371701409306000853
:104DF0002328D780371701408946232AD7803E874A
:104E00007D177DFF37170140032687801982058AA9
:104E100089462328D7803E877D177DFF13573500AD
:104E2000058B6307071037170140930600082328F6
:104E3000D780371701408946232AD7803E877D17C0
:104E40007DFFB716014003A786801983058B89482B
:104E500023A81681BE86FD16FDFE0A0733670701EB
:104E6000598E0547630DE60C371701408546232808
:104E7000D7808946232AD7803E877D177DFF371745
:104E8000014089462328D780FD17FDFFB717014051
:104E9000094723AAE78083A781663E877D177DFFA8
:104EA0003717014089462328D7803E877D177DFF2D
:104EB000371701408546232AD7808946232AD78081
:104EC0003E877D177DFF3717014089462328D7800D
:104ED0003E877D177DFF3717014093060008232882
:104EE000D7801375050819C123A6016683C601671B
:104EF0007D58371501408945FD16638F0627232A03
:104F0000B5803E877D177DFF2328B5803E877D17BE
:104F10007DFFDDB7B71701401307000823AAE7801C
:104F200079B53717014093060008232AD780D9B5F1
:104F30003717014093060008232AD780DDBD137779
:104F40002500630607107D43B71801409388088049
:104F5000094EF28E23AAD8013E877D177DFF03A755
:104F600088001983058B23A8C8013E887D18E31F9C
:104F700008FE7E07558F935617007D13E31C03FC34
:104F8000138741668348A701383FB388E840054747
:104F90006383E808371701400948232A07813E87C1
:104FA0007D177DFF37180140032788801983058B03
:104FB0000943232868803E887D18E31F08FEF918FE
:104FC000638708023713014013030380094EF28EF2
:104FD000232AD3013E887D18E31F08FE2328C3013E
:104FE0003E887D18E31F08FEFD18E39308FE37187E
:104FF00001408548232818818948232A18813E8842
:105000007D18E31F08FE37180140894823281881BE
:10501000FD17FDFF3DA037170140054823280781F4
:105020000948232A07813E877D177DFF37180140F5
:10503000032788801983058B894823281881FD1749
:10504000FDFFE38505E47E07558F98C181B58C414E
:105050007D4837170140130707809308000809436C
:105060001A8E0DA0232A1701232AC701BE86FD161A
:10507000FDFE23286700BE86FD16FDFE85817D1896
:105080006308080093F61500F1DE23281701E9BF35
:1050900013874166342F383F998E0547638AE608A7
:1050A0008589C1C1B71701401307000823A8E7800D
:1050B000B7170140094723AAE78003A78166BA878B
:1050C000FD17FDFFB7170140894523A8B780BA87B0
:1050D000FD17FDFFF9169DC2B715014093850580A8
:1050E0000948C28823AA1501BA87FD17FDFF23A826
:1050F0000501BA87FD17FDFFFD16EDF6B717014054
:10510000854623A8D780894623AAD780BA87FD176A
:10511000FDFFB7170140894623A8D7807D177DFF83
:10512000B5B3B71701401307000823AAE78049B7B2
:105130003717014085462328D78085899DC53717B5
:105140000140930600082328D7803717014089467D
:10515000232AD7803E877D177DFF37170140894678
:105160002328D780FD17FDFF15B33717014093069D
:105170000008232AD780D1BF1375F60F8280130849
:10518000F5FF29C903A5816681460147371601400D
:1051900013060680854E8948468E7D5315A0232A26
:1051A000D601232AC601AA87FD17FDFF2328160171
:1051B000AA87FD17FDFF0583FD167D18630C6800A7
:1051C00081E698218505A14693771700E9DB23281E
:1051D000D601C1BF82809376F503CDC6137505084D
:1051E00001CD214581453718014013080880094346
:1051F0001A8E9388416629A8D9EA82809306000412
:10520000CDB7930716000CA295CE3E86AA85214500
:10521000232AC80183A748003E877D177DFF032707
:105220008800058B23286800FD17FDFF85819317F3
:105230007700DD8D7D15FD1669D5F9FAB3D7A50088
:105240001CA28280828023AA650023AA1501AA8756
:10525000FD17FDFF23A80501AA87FD17FDFF0582A5
:105260007D17FD1609CB99C693771600E9DF23A8B1
:105270006500E1BF828091C603460E00050E2147FE
:10528000E5B782801375050835F993060004138E7F
:105290001500902103A581662147B715014093852C
:1052A000058005430948C288C1B783C75166638634
:1052B000073AB7170140054723A8E780094723AA03
:1052C000E78023A8E78093771500638C0716B7174C
:1052D0000140054723A8E780B7170140094723AAE3
:1052E000E78023A8E7809357150013F717006300A2
:1052F00007163717014085462328D7803717014006
:105300008946232AD7802328D78013572500BA97A8
:10531000058B630407143717014085462328D7807F
:10532000371701408946232AD7802328D780AA9798
:105330009356350013F7160063070712371701401D
:1053400005462328C780371701400946232AC7800E
:105350002328C78013070780B697858B638B0710B8
:10536000BA87054798CBB7160140094723AAE680BC
:1053700023A8E680054623AAC68023AAE68023A8A0
:10538000E68023A8C68023AAE68023A8E68023A877
:10539000C68083A70680C19B93E7870023A0F68081
:1053A00083C7C16791CB3717014013070780894630
:1053B00054CB14CBFD17EDFF371701408946232A44
:1053C000D780032887802328D780232AD780832764
:1053D00087802328D780232AD78003268780232805
:1053E000D78013F717000607937716008A075D8F9B
:1053F000937718005D8F85476303F7089307E7FFEE
:10540000F59B6386071C83C7C16793871702B7168E
:105410000140938606800946D0CA90CAFD17EDFF69
:10542000B7160140854523AAB68083A70680C19B95
:1054300093E7370023A0F68023A8B6801375F70FF3
:105440008280B7170140054723AAE78071B5371757
:1054500001408546232AD78055B537170140854638
:10546000232AD78075BD371701400546232AC780F8
:10547000D9BDB7170140054723AAE780EDB593775B
:105480002500DDCF13080002814681483716014010
:10549000130606800943232A66001C46858B2328B1
:1054A0006600BE988582FE07DD8E7D18E31508FE36
:1054B000B7170140094623AAC78003A8878023A8FD
:1054C000C780B3C8080193F8180063830800214718
:1054D00091C194C183C7C16791CBB7160140938630
:1054E00006800946D0CA90CAFD17EDFFB7160140E5
:1054F000054623AAC68083A70680C19B93E7370091
:1055000023A0F6801375050819C123A6016683C779
:10551000016799CFB7160140054623AAC680B71682
:105520000140938606800946D0CA90CAFD17EDFF58
:10553000B7170140854623A8D7801375F70F8280DF
:1055400083C7C16791CBB716014093860680094691
:10555000D0CA90CAFD17EDFFB7160140054623AA31
:10556000C68083A70680C19B93E7370023A0F680FF
:105570009C41130600028145938606800543094835
:1055800019A823AA660023AA060123A80601BE952E
:1055900085837D1601CA93F81700E38408FE23A8CB
:1055A0006600D5B7858991CDB7170140854623A8F8
:1055B000D780B7170140894623AAD78023A8D78070
:1055C00091B7B7170140854623AAD780DDB783C7B7
:1055D000D16799CF9377250081CF93071002B71633
:1055E0000140938606800946D0CA90CAFD17EDFF98
:1055F00083C7C16791CBB7160140938606800946E1
:10560000D0CA90CAFD17EDFFB7160140054623AA80
:10561000C68083A70680C19B93E7370023A0F6804E
:1056200083C7D1679DC309890DE1B717014085463E
:1056300023AAD78093071002B716014093860680ED
:105640000946D0CA90CAFD17EDFFB717014085463D
:1056500023A8D7801375F70F8280B717014005473D
:1056600023A8E780094723AAE78083A781663E87AE
:105670007D177DFF3717014089462328D7803E8755
:105680007D177DFF13771500630A07263717014042
:1056900085462328D780371701408946232AD7809B
:1056A0003E877D177DFF3717014089462328D78025
:1056B0003E877D177DFF135715009376170063858E
:1056C0000624B7160140054623A8C680B716014038
:1056D000094623AAC680BE86FD16FDFEB716014008
:1056E000094623A8C680BE86FD16FDFE93562500FA
:1056F0003697858A63800622B7160140054623A89F
:10570000C680B7160140094623AAC680BE86FD168C
:10571000FDFEB7160140094623A8C680BE86FD16C9
:10572000FDFE2A971356350093761600638A061EEF
:10573000B7160140054823A80681B716014009485D
:1057400023AA0681BE86FD16FDFEB7160140094854
:1057500023A80681BE86FD16FDFE3297058B6307E2
:10576000071C3717014085462328D780371701408B
:105770008946232AD7803E877D177DFF3717014052
:1057800089462328D7803E877D177DFF3717014044
:105790008546232AD7808946232AD7803E877D17CE
:1057A0007DFF3717014089462328D7803E877D1724
:1057B0007DFF3717014085462328D7808946232A55
:1057C000D7803E877D177DFF371701408946232804
:1057D000D780FD17FDFF3717014085462328D78066
:1057E00083270780C19B93E787002320F78083C727
:1057F000C1678DC703A68166B716014093860680F0
:105800000948C28823AA160132877D177DFF23A885
:10581000060132877D177DFFFD17EDF7B7170140B1
:10582000094723AAE78083A781663E877D177DFF0E
:1058300037170140032687801378160089462328EE
:10584000D7803E877D177DFF371701408946232A81
:10585000D7803E877D177DFF37170140032687805D
:10586000058A89462328D7803E877D177DFF9316BA
:105870001600371701400946232AC7803E877D1747
:105880007DFF3717014003268780058A8948232832
:1058900017813E877D177DFF0A06558E3366060108
:1058A0008546630BD6081307E6FF759B630407263E
:1058B00083C6C16793861602B7150140938505809C
:1058C00009452A8823AA05013E877D177DFF88C9DF
:1058D0003E877D177DFFFD16F5F63717014085459C
:1058E000232AB78083270780C19B93E737002320B3
:1058F000F7802328B7801375F60F82803717014091
:105900008546232AD78041BBB7160140054623AA06
:10591000C6806DBBB7160140054623AAC680D5B325
:10592000B7160140054823AA068101BD371701407B
:105930008546232AD7801DBD93762500DDCE3A8883
:10594000130E00023713014013030380894E768F34
:10595000232AE301BE86FD16FDFE83268300858A89
:105960002328D301BE88FD18E39F08FE36971358FD
:105970001800FE0633E806017D1EE31B0EFCB71679
:105980000140894823AA1681BE86FD16FDFEB71682
:10599000014083A8868093F81800094323A86680F5
:1059A000FD17FDFF058B63031701214699C123A055
:1059B000050103C7C1670DC783A58166B7160140FE
:1059C000938606800948C28823AA1601AE87FD1770
:1059D000FDFF23A80601AE87FD17FDFF7D176DF7BC
:1059E000371701408546232AD78083270780C19B2C
:1059F00093E737002320F780C1A003C8C167630580
:105A00000802B71801409388088009431A8E23AA18
:105A1000C801BE86FD16FDFE23A86800BE86FD16E1
:105A2000FDFE7D18E31508FEB7160140054823AAC0
:105A3000068183A70680C19B93E7370023A0F680E9
:105A40009C4183A8816613080002B7150140938525
:105A500005800543094EF28E15A023AA650023AAEE
:105A6000D501C686FD16FDFE23A8C501C686FD1616
:105A7000FDFE3E9785837D186308080093F61700A6
:105A8000E9DE23A86500E1BF058B3DCFB7170140D4
:105A9000054723A8E780B7170140094723AAE780F5
:105AA00083A781663E877D177DFF371701408946B2
:105AB0002328D780FD17FDFF1375050819C123A6FC
:105AC000016603C701670DCBB7170140854623AABE
:105AD000D78083A58166B716014093860680094565
:105AE0002A8823AA0601AE87FD17FDFF88CAAE8764
:105AF000FD17FDFF7D1775F7B7170140054723A870
:105B0000E7801375F60F8280B7170140054723AA77
:105B1000E78051B703C7D16705CB137725000DC7C1
:105B200093061002B7150140938505800948C28885
:105B300023AA15013E877D177DFF23A805013E8717
:105B40007D177DFFFD16EDF683C6C1679DC2B715B3
:105B50000140938505800948C28823AA15013E8724
:105B60007D177DFF23A805013E877D177DFFFD166C
:105B7000EDF6371701408546232AD7808327078013
:105B8000C19B93E737002320F78083C7D16795CF68
:105B9000937725009DEBB7170140054723AAE780BF
:105BA00083A5816613071002B7160140938606800D
:105BB00009452A8823AA0601AE87FD17FDFF88CA7A
:105BC000AE87FD17FDFF7D1775F7B7170140054735
:105BD00023A8E7801375F60F8280B3C7A5008D8BCD
:105BE0003307C50081E78D4763EDC700AA87637E51
:105BF000E508942185078505A38FD7FEE3EBE7FE33
:105C0000828093763500AA8789CA94218507850505
:105C1000A38FD7FE93F63700C5BF9376C7FF1386D1
:105C200006FE63F0C70683A3050083A2450083AF89
:105C3000850003AFC50083AE050103AE450103A394
:105C4000850183A8C5019385450223A0770003A899
:105C5000C5FF23A2570023A4F70123A6E70123A829
:105C6000D70123AAC70123AC670023AE170193878E
:105C7000470223AE07FF75B790419107910523AE08
:105C8000C7FEE3EBD7FEE3E6E7F682800902620097
:105C900003010000640904000002FF00000407057E
:105CA000010240000107058102400001080B0102CA
:105CB00002020100090401000102020100052400A2
:105CC000100105240100020424020005240601023B
:105CD0000705820308000A09040200020A00000006
:105CE0000705830240000007050302400000000092
:105CF0001201010200000040861A21701001010209
:105D0000030100000600FF0901A101190129401546
:105D10000026FF0075089540810019012940910077
:105D2000C00000002403580056002D004C006900FC
:105D30006E006B00200043004D00530049005300EB
:105D40002D004400410050002403580056002D004F
:105D50004C0069006E006B00200043004D005300B2
:105D6000490053002D004400410050001203580028
:105D7000490056004E00310039003800370000005D
:105D80004A0C0000620C0000740C0000820C000041
:105D9000A00C0000C20C0000A42C0000602D00002C
:105DA000C42D0000A82E000030330000583300003E
:105DB000F43B0000D43F00003C3F00003A2F0000BD
:105DC0005A2F0000D43F0000D43F0000D43F000011
:105DD000D43F0000D43F0000662F0000C030000018
:105DE0002C31000052310000263200008C320000BD
:105DF000E8320000D43F0000D43F0000D43F000050
:105E0000D43F0000D43F0000D43F000070310000B8
:085E100056312E3200000000A3
:105E1800050F2100011C100500DF60DDD88945C78A
:105E28004C9CD2659D9E648A9F00000306A60034A0
:105E3800000000000A00000000000306A600080099
:105E4800020000009C001400030057494E555342BD
:105E580000000000000000000000800004000100B5
:105E68002800440065007600690063006500490069
:105E78006E007400650072006600610063006500D2
:105E8800470055004900440000004E007B004300D5
:105E980044004200330042003500410044002D0018
:105EA80032003900330042002D003400360036003D
:105EB80033002D0041004100330036002D00310031
:105EC80041004100450034003600340036003300FC
:105ED8003700370036007D00000000001A0330004C
:105EE8003100320033003400350036003700380006
:105EF80039004100420000008806000068020000E6
:105F08006A0200002C1700002C1700002C17000054
:105F18002C170000E80500002C1700007E02000086
:105F28002C1700002C1700002C1700002C1700005D
:105F3800B8070000160800008C070000AA06000039
:105F4800E006000062070000AC0600009A0A0000A4
:105F5800AA0A0000BA0A0000000000004000000081
:105F6800FC010020040000006C5D0000120000002D
:105F7800485D000024000000CC0000201A0000004A
:105F8800245D0000240000002C170000900600008B
:105F98002C1700002C1700002C170000A806000082
:105FA8002C170000A60600009E0600000000000056
:105FB80001020304010203040607080900000000A7
:105FC800000000202100000024000020A60000009E
:105FD800010000008C5C000062000000F05C000022
:105FE800120000000F010000E95C00000900000039
:105FF800045D00001D000000010000000044950839
:106008000204060800C20100000008000403090495
:08601800322E312E3000000091
:00000001FF
